:020000040000FA
:0200000056297F
:08000800F000030EF200830179
:100010000408F1008C1C31288C10BB20B60B16286C
:100020001030B6003708B5003808850035080319C8
:100030001C288616B5031D288612B903390FBA0A83
:10004000BA0339083A04031D31280030BA001430CD
:10005000B9004608A2004708A30033143311061361
:1000600033160C1D4E280C11171C3C281508A00037
:100070001608A10017104E2817141508A20016081C
:10008000A3002008A2022108031C210AA3023314A2
:10009000331506170030BA001430B9007108840017
:1000A000720E8300F00E700E09008A01820701347F
:1000B0000134013401340134013401340234023496
:1000C000023402340234023403340334033403347C
:1000D0000334033404340434043404340434043462
:1000E0000534053405340534053405340534063447
:1000F000063406340634063406340734073407342D
:100100000734073407340834083408340834083412
:1001100008340934093409340934093409340934F8
:100120000A340A340A340A340A340A340B340B34DD
:100130000B340B340B340B340C340C340C340C34C3
:100140000C340C340D340D340D340D340D340D34A9
:100150000D340E340E340E340E340E340E340F348F
:100160000F340F340F340F340F3410341034103474
:1001700010341034103400308A003F088207C2283F
:10018000D428EF28061CD1280800BF018613EE30C2
:10019000BD000230BE00FA30C0000030C100B31014
:1001A00008000130BF0008000618E2288617B318BF
:1001B0000800BD033D0FBE0ABE033D083E040319FF
:1001C000B3140800B31CC5280230BF00F230C400CD
:1001D0000530C500F230C8000530C9000800061C13
:1001E0002029C003400FC10AC10340084104031D78
:1001F0000029FA30C0000030C1000608803A8600AD
:10020000331C0800331045082302031D0929440844
:10021000220203180F292208C4002308C500490838
:100220002302031D152948082202031C1B2922084A
:10023000C8002308C9002208C6002308C700080018
:100240004808B1004908B2001530B1020030031C63
:100250000130B2024608B1024708031C470AB20245
:100260004608AF004708B0001530AF020030031C4D
:100270000130B0024408AF024508031C450AB00231
:100280003108A8003208A900C830A600A70135220D
:100290002408CA002F08A8003008A900C830A6000A
:1002A000A70135222408CB00B315C5288301BF015F
:1002B000B3018501860107309F0083160A30810053
:1002C0008501860106148615051685160C158C14F5
:1002D000FA3092008301013090000530970005301C
:1002E00092008617C520B301B4010830F50008302C
:1002F000F3004430F40074088400831673089B00F4
:100300001C141A0883128000F30AF40AF50B7B29E7
:10031000A201A3010030BA001430B900B701851A58
:10032000A5290830F5000030F3004430F4007408CB
:100330008400831673089B001C141A088312800023
:10034000F30AF40AF50B9729B3150B178B178613CD
:100350006400B318A829B319B729331AB22933187E
:10036000D729A8293312B701B5018612A829B311DC
:100370000830F5004430F3000830F4008C137308A3
:100380008400000883169A0074089B001C158B13C8
:1003900055309D00AA309D009C148B171C118312B0
:1003A0008C1FD029F30AF40AF50BBE29A8293310B3
:1003B00049082302031DDE2948082202031CE42900
:1003C0004808A2004908A30045082302031DEA29A2
:1003D000440822020318F0294408A2004508A3009B
:1003E0002208AD002308AE004608AD024708031CF2
:1003F000470AAE02031C012A0430AC004A08AB00D5
:100400000C2A0830AC004B08AB00AD09AE092D0F2B
:10041000AE03AE0AAD002E0400302E02031D122AD8
:1004200015302D02031C232A1530AD020030031CA9
:100430000130AE022D08A8002E08A9002B08A60046
:10044000A70135222C2A051E282A8612B701A829C1
:100450000030AC00C730A4000310240C8B135520CF
:10046000B7008B172C08B800A8290630AA00031083
:10047000A80DA90DAA0B372AA401A5012608270457
:100480000319FF340130AA00A71B4B2AAA0A031044
:10049000A60DA70D442A0310A40DA50D2608A80239
:1004A0002708031C270AA90203185D2A2608A807A3
:1004B00027080318270AA9075E2A2414AA03031988
:1004C000652A0310A70CA60C4B2A0310A80DA90D32
:1004D0002608A8022708031C270AA902031C0800F3
:0C04E000240FA503A50AA4002504003485
:02400E004D3F24
:1042000030000400F2000500B400070090009000A8
:1042100030000400F2000500B40007009000900098
:00000001FF
